:100000000C94C9050C94E4050C943F170C946317E9
:100010000C94E4050C949C120C94E4050C94E405F7
:100020000C94E4050C94E4050C949D0A0C94E405EE
:100030000C94E4050C94E4050C94E4050C94E4059C
:100040000C94E4050C94E4050C94E4050C94E4058C
:100050000C94E4050C94E4050C946214415652206F
:10006000427574746572666C792047434300546925
:100070006D6500436C6F636B0041646A7573742037
:10008000436C6F636B004368616E676520436C6F00
:10009000636B20466F726D6174004461746500414A
:1000A000646A7573742044617465004368616E67A7
:1000B00065204461746520466F726D6174004D75F2
:1000C000736963004E616D6500456E746572206EE4
:1000D000616D650054656D7065726174757265005F
:1000E000566F6C74616765004C69676874004F7087
:1000F00074696F6E7300446973706C617900416458
:100100006A75737420636F6E7472617374004272E7
:100110006F777365207365676D656E747300446FE8
:10012000776E6C6F6164204E616D6500426F6F7415
:100130006C6F6164657200506F77657220536176F1
:1001400065204D6F6465004175746F20506F776551
:10015000722053617665000A045A0A020B0A0514DC
:100160000B030A14040A14021514030A14052815B3
:10017000041B15021615031415051B170419170186
:10018000181703161705191904171901241903164E
:100190001905171B04151B021C1B03141B05151D39
:1001A000041F1D011E1D031C1D051F1F041D1F0113
:1001B000201F031C1F051D28041428022A28030AD7
:1001C00028053229022A2903283204283202333230
:1001D000030A32053C35043735013635033335051E
:1001E000373704353701383703333705353C0432A8
:1001F0003C023D3C030A3C054646043C4602474659
:10020000030A46055050044650025150030A500557
:100210005A5A04505A025B5A030A5A050A5B04628E
:100220005B025C5B035A5B055E5C015D5C035B5ECD
:10023000045B5E025F5E035A5E056060045E6002FE
:100240006160035A60056262046062026362035A7D
:1002500062055B0000000A5C0000000B0000C407A0
:10026000146E0000001573000000160000B20E1797
:1002700079000000180000260F19860000002400F5
:10028000003A101B9A0000001C000080101D9F0007
:1002900000001E00002F111FAB00000020000058BE
:1002A0001228BE0000002A00009D0C2B00003C0D0F
:1002B00032C40000003300005A0835C9000000377E
:1002C0001E010000360000AE08380000B0093CD422
:1002D0000000003D0000F21946E000000047000069
:1002E000291A50E80000005100004C1A5AEE000094
:1002F000005BF60000005CFE0000005D0000AE1335
:100300005E2C0100005F0000FE0660370100006106
:1003100000001C0762470100006300003D07000069
:100320000000004A756D7020746F20626F6F746CEE
:100330006F6164657200507265737320656E7465D9
:100340007220746F20736C656570004F6666004F95
:1003500066660077616974696E6720666F722069EE
:100360006E707574206F6E205253323332005465B4
:100370007374004C65667400557000526967687448
:1003800000446F776E00536F756E64004C434420D9
:1003900074657374004572726F722054656D706578
:1003A000726174757265004572726F7220566F6C5F
:1003B00074616765004C69676874004572726F729A
:1003C0002044617461666C617368004675722045F3
:1003D0006C69736500030008007B01080092010846
:1003E000007B010800920108007B010800FA010867
:1003F00000AA010800DE010400380208000100081C
:1004000000BC030800F602080038020400FA0108E4
:100410000001000800F60208005A020800FA010470
:1004200000DE01080001000800F60208007B010858
:1004300000920108007B010800920108007B01087E
:1004400000FA010800AA010800DE010400380208D1
:100450000001000800BC030800F60208003802048E
:1004600000FA01080001000800F6020800DE010899
:1004700000FA0104003802000001005475726B6537
:1004800079206D617263680003001000A4021000FF
:10049000F602100024031000F60204007E02100091
:1004A000380210007E021000A40210007E02040038
:1004B000FA011000DE011000FA011000180210000D
:1004C000FA011000520110007B011000920110008F
:1004D0007B011000520110007B01100092011000FE
:1004E0007B0104003F0108007B0108003F01200060
:1004F000AA0120007B011000520108007B010800C6
:10050000AA0108007B012000AA0120007B01100045
:10051000520108007B010800AA0108007B012000AD
:10052000AA0120007B011000520108007B01080095
:10053000AA010800C3010400FA01000001004D698E
:100540006E7565740002000400AA0108007E0208AE
:100550000038020800FA010800DE010400AA0104C4
:10056000007E0204007E0204007B010800DE010818
:1005700000AA0108007B010800520104003F0104A9
:10058000007E0204007E020400DE010800AA0108C9
:1005900000DE010800FA01080038020400FA010830
:1005A00000DE010800FA010800380208007E02049B
:1005B00000A40208007E02080038020800FA0108C0
:1005C000007E020400FA010200380200000100412E
:1005D000756C64204C616E672053796E6500030072
:1005E00004003F010200EF000800EF000400EF00EC
:1005F0000400BE000200D5000800EF000400D50092
:100600000800BE000800D5000200EF000800EF005F
:100610000400BE0004009F0002008E0008000100DC
:1006200004008E0002009F000800BE000400BE000F
:100630000400EF000200D5000800EF000400D50020
:100640000800BE000800D5000200EF0008001C01F1
:1006500004001C0104003F010200EF00040001003F
:1006600000000100536972656E65310000002000D2
:10067000900120008D0120008A01200087012000C8
:1006800084012000810120007E0120007B012000E8
:100690007801200075012000720120006F01200008
:1006A0006C01200069012000660120006301200028
:1006B000600120005D0120005A0120005701200048
:1006C00054012000510120004E0120004B01200068
:1006D0004801200045012000420120003F01200088
:1006E0003C012000390120003601200033012000A8
:1006F000300120002D0120002A0120002A012000C5
:100700002D0120003001200033012000360120009F
:10071000390120003C0120003F012000420120005F
:1007200045012000480120004B0120004E0120001F
:100730005101200054012000570120005A012000DF
:100740005D0120006001200063012000660120009F
:10075000690120006C0120006F012000720120005F
:1007600075012000780120007B0120007E0120001F
:100770008101200084012000870120008A012000DF
:100780008D012000900100000100536972656E65C3
:10079000320003000400DE0104003F0100000100FC
:1007A00057686973746C650000002000C800200061
:1007B000C3002000BE002000B9002000B4002000CB
:1007C000AF002000AA002000A5002000A00020000B
:1007D0009B00200096002000910020008C0020004B
:1007E00087002000820020007D002000780020008B
:1007F000730020006E0020006900200064000800E3
:1008000001002000C8002000C3002000BE0020001E
:10081000B9002000B4002000AF002000AA00200092
:10082000A5002000A00020009B00200096002000D2
:10083000910020008C002000870020008200200012
:100840007D0020007D002000820020008700200025
:100850008C00200091002000960020009B002000CA
:10086000A0002000A5002000AA002000AF0020006A
:10087000B4002000B9002000BE002000C30020000A
:10088000C80000000000D50388044505DE056C069D
:100890009207A8070000504C4159494E4700444474
:1008A0004D4D5959004D4D444459590059594D4DDC
:1008B0004444000405020300010405000102030092
:1008C0000102030405323448003132480031324815
:1008D00000323448003234480031324800510A8036
:1008E0002A0000000A510A000059551801111E1172
:1008F0001B500B411B411F1101511F511B000000D8
:100900000000000000000000000000510F9139417C
:10091000149131411E410E411D500F802010154889
:10092000864014780570855115510E5195518E21D0
:100930009081205015484450C528C02820095000F7
:1009400000000000000000000009090909090A0A66
:100950000B0801080108010801080110021002201B
:100960000426031C0312030703FD02F202E702DC64
:1009700002D002C502B902AD02A102950289027C31
:10098000027002630257024A023E02320225021935
:10099000020C020002F401E801DC01D001C401B83C
:1009A00001AD01A20196018C01810176016C016209
:1009B0000158014E0144013B013201290120011778
:1009C000010F010701FF00F700F000E900E100DB83
:1009D00000D400CD00C700C100BB002F0339034283
:1009E000034B0353035C0364036C0373037B0382B5
:1009F0000388038F0395039B03AA03A703A403A102
:100A0000039E039B039803940391038D038A03863B
:100A10000382037E037B03770372036E036A03661C
:100A20000361035D03580353034F034A0345034027
:100A3000033B03360330032B03260320031B03155C
:100A4000030F030A030403FE02F802F202EC02E6BB
:100A500002DF02D902D302CC02C602BF02B902B23F
:100A600002AC02A5029E02970291028A0283027CD6
:100A70000275026E02680261025A0253024C02457C
:100A8000023E0237023002290222021B0215020E28
:100A90000207020002F901F201EC01E501DE01D8D2
:100AA00001D101CB01C401BE01B701B101AA01A46A
:100AB000019E01980192018C01860180017A0174E6
:100AC000016E01680163015D01580152014D01474A
:100AD0000142013D01380133012E01290124011F8A
:100AE000011A01150111010C0108010301FF00FBAE
:100AF00000F600F200EE00EA00E600E200DE00DBB5
:100B000000D700D300CF00CC00C800C500C200BE93
:100B100000BB00350060008000B0001D013D015A9F
:100B2000017A019701B901DA01F901160240026D5B
:100B3000028202A202EF023203B003F2031D5A3412
:100B400040E17A34406ABC344091ED34407D3F3519
:100B500040A47035402DB23540F2D23540B6F33561
:100B6000403F353640666636408D97364017D93659
:100B700040643B3740EE7C374014AE37409EEF3741
:100B800040B0723840E926394021B03A4093183CD1
:100B9000400011241FBECFEFD4E0DEBFCDBF11E077
:100BA000A0E0B1E0EAEFF6E302C005900D92AE35A9
:100BB000B107D9F711E0AEE5B1E001C01D92AE3F3B
:100BC000B107E1F70C94E6050C940000CFEFD4E0F8
:100BD000DEBFCDBFCC248AE0D82ED0929C010CE59C
:100BE00010E0EE24FF240E94DA067894C0915F01A1
:100BF000CC2309F048C00115110549F061E0C80196
:100C00000E942C138C2F0E949D1300E010E00E9484
:100C1000BB17682FE114F10471F0F701099511C0B9
:100C2000F901E95AFD4F05911491F901E75AFD4F79
:100C3000E590F49028C0882329F080919C010E94BF
:100C4000B006D82E80919C01D816E9F0D0929C0174
:100C500040E065E0E6E5F2E084918823A1F0469F5C
:100C600090011124F901EA5AFD4F949180919C0161
:100C70009817B1F24F5F469FF0011124EA5AFD4FD9
:100C80008491882361F780910101882371F090910C
:100C9000890180910001981740F08AE080939C01BF
:100CA0001092890181E080935F011F9904C01E9911
:100CB00002C00E94400B93B19095907D8CB18095BD
:100CC0008C70982B9C1521F0C92E10925E010BC0E0
:100CD000992349F080915E01813011F40E948717B9
:100CE00083E080935E0180916001882369F58091A3
:100CF0006101882349F590915F01992329F0809142
:100D0000E4008F778093E40083B7817F866083BFA0
:100D100085B7816085BF889585B78E7F85BF99230C
:100D2000E9F01E991BC010925F0140E0ECEEF0E08C
:100D300011924F5F4431E0F38091E400806880932A
:100D4000E4000E94BB170AC083B7817F83BF85B7C9
:100D5000816085BF889585B78E7F85BF13BE46CFDE
:100D6000582F982F40E023E0E7E5F1E084918823B5
:100D7000F1F0429F90011124F901E95AFE4F84914C
:100D8000851759F4F901E85AFE4F8491861729F422
:100D9000F901E75AFE4F94910AC04F5F23E0429F4A
:100DA000F0011124E95AFE4F8491882311F7892F0D
:100DB000992708950E94F70790E89093610083E0D7
:100DC0008093610090BF87E080937F008FE085B9BA
:100DD00080EF8EB9259A2D9A0E9427170E94730ED4
:100DE0000E94850A8CE090E00E94640A0E949A1595
:100DF0000E94AC15289A0E940D140895982F809196
:100E00000201882341F01092020161E083E293E045
:100E10000E942C130EC0913021F488E18093600071
:100E2000FFCF933031F481E0809302018EE590E0B2
:100E300008958FE590E00895982F8091030188230D
:100E400041F01092030161E086E393E00E942C13CD
:100E500011C0913039F490935F01909303018AE0BF
:100E600090E00895933031F481E08093030180E6AF
:100E700090E0089581E690E00895EF92FF920F933D
:100E80001F93CF93F0900401FF2069F010920401AA
:100E900080910101882319F08091000134C061E044
:100EA0008BE493E029C0813029F48093040182E629
:100EB00090E054C0843059F4809100018B5F80939E
:100EC00000018B35E0F08AE58093000145C0853054
:100ED00009F042C080910001882319F08550809369
:100EE000000180910001853050F4F0920101F092F0
:100EF000000161E08FE493E00E942C132DC091E08B
:100F0000E92EE09201010E94C717C82F082F0F7029
:100F1000005DC295CF70C05D6DE480E00E948B13D0
:100F200069E481E00E948B136EE482E00E948B13DF
:100F300060E283E00E948B136C2F84E00E948B138D
:100F4000602F85E00E948B1360E086E00E948B1387
:100F500060E081E00E94A01383E690E0CF911F91B2
:100F60000F91FF90EF90089501972FEF8F3F920719
:100F700051F020E000002F5F2D37E0F301972FEFB5
:100F80008F3F9207B1F70895982F8091050188232C
:100F900019F11092050162E580E00E948B1365E46F
:100FA00081E00E948B1366E582E00E948B1360E370
:100FB00083E00E948B1366E384E00E948B1361E35D
:100FC00085E00E948B1360E086E00E948B1360E056
:100FD00081E00E94A01308C0933031F481E0809337
:100FE00005018AE090E008958BE090E00895CF93AA
:100FF000C0E080E88093610083E080936100C0934B
:10100000700088E08093B60088EC8093B300C093B2
:101010006E0081E0809381008093B0008091B600E3
:10102000282F3327217030708091B6009927847063
:101030009070282B392B232B89F788EE93E00E94A0
:10104000B407F8948FEF86BB87BB1092850010928F
:1010500084001092B20087B38823E9F310928100D4
:10106000789486B3882319F02FEF3FEF0AC0909150
:10107000840080918500282F3327322F2227290FC3
:10108000311D88E12B36380724F0809166008150AD
:1010900006C0285E374134F4809166008F5F8093EC
:1010A000660001C0C1E081E080938100CC2349F259
:1010B000CF910895CF93DF93CDB7DEB722970FB6C8
:1010C000F894DEBF0FBECDBF282F80E091E089836A
:1010D0009A8380910601882331F110920601F894D9
:1010E000F999FECF89819A8192BD81BDF89A789451
:1010F00080B5682F772760936201862F81508931F0
:1011000030F01092620181E480939D010EC041E0B5
:1011100051E08DE991E00E946B1561E08DE991E06D
:101120000E945F1310C0223031F481E080930601E9
:1011300085E390E00AC0233031F481E0809306011A
:1011400082E390E002C083E390E022960FB6F89429
:10115000DEBF0FBECDBFDF91CF9108951F93CF9318
:10116000DF93CDB7DEB722970FB6F894DEBF0FBE80
:10117000CDBF182F80E091E089839A838091070189
:10118000882391F041E051E0609162018DE991E0A6
:101190000E946B1580916201882319F08150809321
:1011A00062011092070155C0909162019093630112
:1011B00085E080936A01382F492FE92FFF27E356F6
:1011C000FE4F2081822F80528B3540F49F3F31F0BB
:1011D000E32FFF27EC59FE4F208306C0E32FFF27A4
:1011E000EC59FE4F80E280833150942F91503F3F65
:1011F00019F730936A01909363016091640180E074
:101200000E948B136091650181E00E948B136091B5
:10121000660182E00E948B136091670183E00E9467
:101220008B136091680184E00E948B1380916901A7
:101230008068682F85E00E948B1360E086E00E9442
:101240008B13112311F00E94AB1360E081E00E9428
:10125000A013112311F00E94AB131430D1F480912C
:101260006201E82FFF27E356FE4F9081292F21507E
:101270002083892F82528F3030F19B53973010F4A6
:1012800089E33BC02B3518F4203208F05DC08AE5B5
:1012900034C01530D1F480916201E82FFF27E35666
:1012A000FE4F9081292F2F5F2083892F80528F300E
:1012B00010F480E322C099539730F0F02B3518F4E6
:1012C000203208F041C080E218C0133041F4809110
:1012D00062018823C9F181508093620135C01230C8
:1012E00071F480916201893178F58F5F809362019A
:1012F000E82FFF27E356FE4F81E4808325C011309D
:1013000019F5209162012F5F20936201E22FFF27E0
:10131000E356FE4F1082F894F999FECF89819A81A5
:1013200092BD81BD20BDFA9AF99A789441E051E0CE
:10133000609162018DE991E00E943B1581E080930C
:10134000070183E390E002C086E390E022960FB6A7
:10135000F894DEBF0FBECDBFDF91CF911F910895EE
:101360001F93CF93DF93CDB7DEB722970FB6F894D4
:10137000DEBF0FBECDBF182F80E091E089839A8336
:10138000809108018823B1F0F89480E8809361008F
:1013900082E080936100789460E083E593E00E94AE
:1013A0002C1310920801109284018091C60081E0F4
:1013B000809361018091C00087FF68C08091C60062
:1013C000909184018D3061F0993108F05FC0E92F70
:1013D000FF27E559FE4F80839F5F9093840156C09D
:1013E000F89480E88093610083E0809361007894B2
:1013F000992309F447C0E92FFF27E559FE4F1082D2
:101400001092840180916B018823A1F09081E92FD3
:10141000FF27DF01A559BE4F8C91E356FE4F808315
:101420009F5FE92FFF27E559FE4F8081882379F7D9
:101430009093840180918401E82FFF27E356FE4FAB
:10144000108281E08093080120916201F894F9995B
:10145000FECF89819A8192BD81BD20BDFA9AF99A09
:10146000789441E051E0609184018DE991E00E941F
:101470003B1580918401809362011092610183E3A6
:1014800090E018C081E0809308010FC0112381F023
:1014900081E080930801F89480E88093610083E004
:1014A0008093610078941092610187E390E002C01C
:1014B00088E390E022960FB6F894DEBF0FBECDBF52
:1014C000DF91CF911F9108959C01832F99278093DD
:1014D000C5002093C40082E08093C00080E1809327
:1014E000C10086E08093C2000895982F8091C000CB
:1014F00085FFFCCF9093C60008958091C00087FFC0
:10150000FCCF8091C6009927089590E0EAEBF1E0C6
:10151000119211929F5F9430D8F390E0E6EBF1E0E6
:101520008FEF81939F5F9430D8F382E080936E00B9
:1015300086E287BD8CE084BD08951F920F920FB69E
:101540000F9211240F931F932F933F934F935F9309
:101550006F937F938F939F93AF93BF93CF93EF93AB
:10156000FF93C0E00AEB11E0D801ED91FD918D01F0
:10157000309709F00995CF5FC430B0F3C0E0E6EBD7
:10158000F1E080818F3F21F0882311F0815080832A
:10159000CF5F3196C430A8F3FF91EF91CF91BF9107
:1015A000AF919F918F917F916F915F914F913F91FB
:1015B0002F911F910F910F900FBE0F901F901895B4
:1015C000AC0120E0EAEBF1E081919191841795075D
:1015D00061F02F5F2430C0F320E0EAEBF1E080817E
:1015E0009181892B29F44083518381E090E0089513
:1015F0002F5F3296243098F380E090E008959C01AC
:1016000040E0EAEBF1E0808191818217930729F4B1
:101610001082118281E090E008954F5F329644304D
:1016200090F380E090E0089590E0E92FFF27EA54DE
:10163000FE4F80819F5F8F3F21F41082892F992771
:101640000895943090F380E090E00895F894E82FA6
:10165000FF27EB54FE4F608378940895F894E82FA9
:10166000FF27EB54FE4F8081789499270895F894D2
:10167000E82FFF27EB54FE4F8FEF80837894089577
:101680001F93CF93DF93C0E0C09370006C2F8EE662
:1016900093E00E942C130E94BB178130E1F760E0B9
:1016A00083E793E00E942C130E94BB178330E1F77D
:1016B00060E088E793E00E942C130E94BB178430FF
:1016C000E1F760E08BE793E00E942C130E94BB17C8
:1016D0008230E1F760E081E893E00E942C130E94E1
:1016E000BB178530E1F760E086E893E00E942C1399
:1016F0000E94BB178130E1F780E88093800081E190
:10170000809381008091810081608093810010929C
:10171000890080E580938800C8ECD0E08D2F992760
:1017200087FD9A9580938700C09386008EE190E0B4
:101730000E94B4072597C436D10584F71092800023
:101740001092810060E08CE893E00E942C131C9BB7
:10175000FECF0E94BB178130E1F78091E400877FC4
:101760008093E40090E0ECEEF0E08FEF81939F5FD8
:101770009431D8F31C9BFECF84E690E00E94B4071E
:101780001C99FECF8091E40088608093E40080E0A3
:101790000E94F8170E940018EC01C45CD140C738C1
:1017A000D105B0F060E085E993E00E942C130E941F
:1017B0005D0C0E94BB17C82F8130D9F70E943818E2
:1017C00060E08C2F0E94A0130E94BB178130E1F7CC
:1017D00081E00E94F8170E940018EC01CA52D14023
:1017E0006797B0F060E087EA93E00E942C130E94B4
:1017F0005D0C0E94BB17C82F8130D9F70E943818A2
:1018000060E08C2F0E94A0130E94BB178130E1F78B
:1018100060E085EB93E00E942C130E94BB1781309F
:10182000E1F782E00E94F8170E9400180E94381821
:10183000000060E081E00E94A0130E94BB1781308D
:1018400099F7289A289810E0C0E0D0E0412FBE0117
:1018500081E00E946E161F5F21961233B8F361E09B
:1018600070E081E00E94BA16289A289860E070E043
:1018700081E090E00E94EB1610E080E00E94A51548
:10188000181761F060E08BEB93E00E942C130E942C
:101890005D0C0E94BB178130E1F703C01F5F12335C
:1018A00060F3289A81E00E94C4070E94BB17813030
:1018B000E1F788E180936000FFCF1F9380E8809379
:1018C000800081E18093810080918100816080931C
:1018D00081001092890080E58093880011E01093C8
:1018E00087008FE38093860082E390E00E94B40734
:1018F000109387008EED809386008CE291E00E9429
:10190000B40710928000109281001F91089580E822
:101910008093800080E180938100809181008160CC
:101920008093810010928900809119018093880032
:101930008EEB9DE00E94E00A0895CF93C82F80911E
:101940001A018823E9F010921A0180918701E82F8B
:10195000FF27EE0FFF1FE75FFE4F61E0808191815F
:101960000E942C1380918701E82FFF27EE0FFF1FA5
:10197000EA57F74F859194919093C3018093C201E8
:10198000C430C1F5809187018823C9F4E1E0E09378
:10199000870180910B0190910C01892B71F02E2F02
:1019A0002F5FE22FFF27EE0FFF1FE75FFE4F8081C3
:1019B0009181892BA9F7209387018091870181501C
:1019C0008093870180918701E82FFF27EE0FFF1F8B
:1019D000E75FFE4F61E0808191810E942C1380912E
:1019E0008701E82FFF27EE0FFF1FEA57F74F85917A
:1019F00094912AC0C53069F5809187018F5F8093EB
:101A00008701E82FFF27EE0FFF1FE75FFE4F808162
:101A10009181892B11F41092870180918701E82F21
:101A2000FF27EE0FFF1FE75FFE4F61E0808191818E
:101A30000E942C1380918701E82FFF27EE0FFF1FD4
:101A4000EA57F74F859194919093C3018093C20117
:101A50000FC0C13029F4C0931A018BE290E00AC094
:101A6000C33031F481E080931A0188E290E002C033
:101A70008AE290E0CF9108951F93CF93182F809121
:101A80001B01882379F010921B01109286010E949D
:101A9000870C61E086E998E00E942C1381E0809336
:101AA00060010DC0C0916001CC2349F48EEB9DE034
:101AB0000E94FF0AC0938000C093810054C014307C
:101AC00041F480911901803510F080E50BC08B5FE7
:101AD00009C0153079F4809119018B3010F486E03B
:101AE00001C08550809319011092890080911901DD
:101AF00080938800113029F580916001882399F046
:101B000010926001809181008E7F809381008EEB26
:101B10009DE00E94FF0A10928000109281002D9A91
:101B200010931B0123C080938501109386010E94AE
:101B3000870C612F86E998E00E942C1310936001B6
:101B400018C01330B1F410926001809181008E7F33
:101B5000809381008EEB9DE00E94FF0A109280002E
:101B6000109281002D9A81E080931B018AE290E01F
:101B700002C08BE290E0CF911F9108950F931F93C5
:101B8000CF93DF9380918601882369F48093850148
:101B9000E091C201F091C3018591949180938801F5
:101BA00081E08093860180918801882309F093C0A9
:101BB00080918501882321F081508093850184C024
:101BC00080918601E82FFF27EE0FFF1F0091C201D1
:101BD0001091C301E00FF11FAF0125913491C82F7F
:101BE000CF5F232B09F44EC0FA012591349180E296
:101BF00090E0B9010E94691B60938501C093860142
:101C000040E050E0EC2FFF27EE0FFF1FE00FF11F29
:101C1000859194918130910509F4AC0120E030E088
:101C20008130910509F49C01422B532B452B21F067
:101C3000809181008E7F03C08091810081608093BC
:101C40008100F89480918601282F3327220F331FBB
:101C5000F801E20FF31F85919491892F990F990B49
:101C6000109285001092840080938700F801E20FA3
:101C7000F31F8591949180938600789480918601DA
:101C80008F5F0DC0C0938601EC2FFF27EE0FFF1F63
:101C9000E00FF11FC591D491CC2321F081E0809316
:101CA000860112C0C0938601C093600180918100BB
:101CB0008E7F809381008EEB9DE00E94FF0AC0938F
:101CC0008000C09381002D9AE091C201F091C30180
:101CD0008591949101C0815080938801DF91CF91CB
:101CE0001F910F91089588EE93E00E94B407F89435
:101CF000809170008E7F8093700088E08093B600A2
:101D00001092B2008091B00085608093B000809105
:101D1000B600282F3327217030708091B6009927A4
:101D200084709070282B392B232B89F78FEF87BB7A
:101D30008091700081608093700078941092C5014A
:101D40001092CA018CE08093C40189E08093C6019F
:101D50008AE08093C90183E090E09093C80180936A
:101D6000C7010895CF92DF92EF92FF920F931F93D6
:101D7000CF93C82E80914101882341F48091C40102
:101D8000E82FFF27E75DFE4F808102C08091C401EC
:101D90000E94C717C82F2FE0D22ED82280E3D80E7A
:101DA000C295CF70C80F8091CA010E94C717082F33
:101DB0009FE0E92EE82280E3E80E02950F70080FFD
:101DC0008091C5010E94C717182F8FE0F82EF122CD
:101DD00080E3F80E12951F70180F6C2F80E00E94A0
:101DE0008B136D2D81E00E948B13602F82E00E9487
:101DF0008B136E2D83E00E948B13612F84E00E9471
:101E00008B136F2D85E00E948B1360E086E00E94AB
:101E10008B1381E00E949D1360E081E00E94A0137B
:101E200083E0C81619F485E190E008C082E0C81686
:101E300019F487E190E002C086E190E0CF911F9114
:101E40000F91FF90EF90DF90CF900895CF92DF92A7
:101E5000EF92FF920F931F93CF93C82E80914E0164
:101E6000882361F08091C40180938B018091CA0125
:101E700080938C018091C50180938D0180914101F7
:101E8000882341F480918B01E82FFF27E75DFE4F07
:101E9000808102C080918B010E94C717C82F5FE02C
:101EA000F52EF82280E3F80EC295CF70C80F80910E
:101EB0008C010E94C717182F4FE0E42EE82280E320
:101EC000E80E12951F70180F80918D010E94C717A0
:101ED000082F3FE0D32ED82280E3D80E02950F7052
:101EE000080F6C2F772780918E01882309F4606892
:101EF00080E00E948B136F2D772780918E018823BD
:101F000009F4606881E00E948B13612F772780912C
:101F10008E01813009F4606882E00E948B136E2D7F
:101F2000772780918E01813009F4606883E00E94F8
:101F30008B13602F772780918E01823009F46068BF
:101F400084E00E948B136D2D772780918E01823063
:101F500009F4606885E00E948B1360E086E00E94CF
:101F60008B1381E00E949D13CC2011F00E94AB13D3
:101F700060E081E00E94A01381E080934E0184E044
:101F8000C81649F480918E01E82FFF27E557FE4FD0
:101F900080818F5F0BC085E0C81651F480918E015F
:101FA000E82FFF27E557FE4F8081815080832FC0A7
:101FB00083E0C81641F480918E01882311F482E0F9
:101FC0000DC081500BC082E0C81659F480918E017B
:101FD000823019F410928E011AC08F5F80938E01A7
:101FE00016C081E0C81699F4F89480918B01809313
:101FF000C40180918C018093CA0180918D018093EE
:10200000C501789410928E0186E190E02BC08091FA
:102010008B018F3F19F487E180938B0180918B01B5
:10202000883110F010928B0180918C018F3F19F450
:102030008BE380938C0180918C018C3310F0109293
:102040008C0180918D018F3F19F48BE380938D017A
:1020500080918D018C3310F010928D0110924E0101
:1020600088E190E0CF911F910F91FF90EF90DF906A
:10207000CF900895CF93C82F80914F01882371F09E
:1020800010924F0160914101613019F485EC98E0A4
:1020900003C061E089EC98E00E942C13C43081F405
:1020A00060914101613029F4109241018DEC98E07A
:1020B00019C081E080934101682F81ED98E012C042
:1020C000C53099F480914101882339F481E08093EF
:1020D0004101682F85ED98E005C01092410161E053
:1020E00089ED98E00E942C1307C0C13029F4C093F9
:1020F0004F0186E190E002C084E290E0CF91089524
:10210000CF92DF92EF92FF920F931F93CF93C82F3E
:102110008091C7010E94C717182FEFE0EE2EE8222A
:1021200080E3E80E12951F70180F8091C9010E947C
:10213000C717082F7FE0D72ED82280E3D80E02954C
:102140000F70080F8091C6010E94C717F82E6FE02C
:10215000C62EC82280E3C80EF694F694F694F69440
:10216000F80E80918A01E82FFF27EE0FFF1FE85B32
:10217000FE4F0190F081E02D8491612F0E948B131E
:1021800080918A01E82FFF27EE0FFF1FE85BFE4FCB
:102190000190F081E02D319684916E2D0E948B1379
:1021A00080918A01E82FFF27EE0FFF1FE85BFE4FAB
:1021B0000190F081E02D32968491602F0E948B1364
:1021C00080918A01E82FFF27EE0FFF1FE85BFE4F8B
:1021D0000190F081E02D339684916D2D0E948B1338
:1021E00080918A01E82FFF27EE0FFF1FE85BFE4F6B
:1021F0000190F081E02D349684916F2D0E948B1315
:1022000080918A01E82FFF27EE0FFF1FE85BFE4F4A
:102210000190F081E02D359684916C2D0E948B13F6
:1022200060E086E00E948B1381E00E949D1360E0D5
:1022300081E00E94A013C33019F48BE190E007C045
:10224000C23019F48DE190E002C08CE190E0CF91B2
:102250001F910F91FF90EF90DF90CF900895FF9224
:102260000F931F93CF93F82E80915001882361F034
:102270008091C70180938F018091C9018093900163
:102280008091C60180939101C0915101CC23C9F482
:1022900080918F010E94C717182F082F0F70005DC3
:1022A00012951F70105D60E28C2F0E948B1360E20C
:1022B00081E00E948B1369E582E00E948B1369E53F
:1022C00035C0C130C9F4809190010E94C717182F02
:1022D000082F0F70005D12951F70105D60E280E0A6
:1022E0000E948B1360E28C2F0E948B136DE482E0BE
:1022F0000E948B136DE41AC0C23019F580919101D0
:102300000E94C717182F082F0F70005D12951F70BD
:10231000105D60E280E00E948B1360E281E00E9429
:102320008B1364E48C2F0E948B1364E483E00E947F
:102330008B13612F84E00E948B13602F85E00E9435
:102340008B1360E086E00E948B1380E00E949D1357
:10235000FF2011F00E94AB1360E081E00E94A01307
:1023600081E08093500184E0F81649F48091510196
:10237000E82FFF27E157FE4F80818F5F0BC085E07C
:10238000F81651F480915101E82FFF27E157FE4FD5
:1023900080818150808332C083E0F81641F48091BF
:1023A0005101882311F482E00DC081500BC082E0FE
:1023B000F81659F480915101823019F410925101AC
:1023C0001DC08F5F8093510119C081E0F816B1F4F0
:1023D000F89480918F0199279093C8018093C70149
:1023E000809190018093C901809191018093C601F1
:1023F0007894109251018CE190E055C080918F014A
:102400008F3F19F483E680938F0180918F0184368A
:1024100010F010928F0180919001882319F48CE0C4
:1024200080939001809190018D3018F081E080932D
:1024300090018091C9018230C9F42091C701309187
:10244000C801C90183709070892B81F4C90164E6C9
:1024500070E00E94691B892B39F4C90160E971E0C1
:102460000E94691B892B11F481E001C080E0882360
:1024700011F0EDE107C080919001E82FFF27E45EA5
:10248000FE4FE08180919101882311F4E093910146
:1024900080919101E81718F481E0809391011092E6
:1024A00050018EE190E0CF911F910F91FF90089520
:1024B000CF93C82F80915201882379F01092520156
:1024C00080918A01E82FFF27EE0FFF1FEE5BFE4F82
:1024D00061E0808191810E942C13C43049F4809185
:1024E0008A01823018F010928A010DC08F5F09C0F6
:1024F000C530B9F480918A01882311F482E001C0CB
:10250000815080938A0180918A01E82FFF27EE0F86
:10251000FF1FEE5BFE4F61E0808191810E942C13D2
:1025200007C0C13029F4C09352018CE190E002C091
:1025300080E290E0CF9108951F920F920FB60F9214
:1025400011242F933F934F935F936F937F938F93B8
:102550009F93AF93BF93EF93FF938091C5018F5FDC
:102560008093C5018C3309F066C01092C50190912B
:10257000CA019F5F9093CA01809189018F5F809308
:1025800089019C3308F457C01092CA018091C4019C
:102590008F5F8093C401883108F44DC01092C4014C
:1025A0008091C6018F5F8093C6014091C90142307E
:1025B000D9F42091C7013091C801C901837090708E
:1025C000892B91F4C90164E670E00E94691B892B94
:1025D00039F4C90160E971E00E94691B892B21F47B
:1025E00081E08093920102C0109292018091C60115
:1025F000282F3327E42FFF27E45EFE4F9081809140
:102600009201890F912D911D82179307A4F491E0F7
:102610009093C601842F890F8093C9018D3058F0A3
:102620009093C9018091C7019091C8010196909340
:10263000C8018093C701FF91EF91BF91AF919F9126
:102640008F917F916F915F914F913F912F910F905B
:102650000FBE0F901F901895FC0180919301882365
:10266000E1F7982F8491882391F0AF01A0EEB1E0BB
:102670009F01F90184918D939F5F2F5F3F4F4F5FC3
:102680005F4FFA018491882311F0993190F3E92F7B
:10269000FF27E052FE4F1082973048F081E0809390
:1026A000CB011092F90183E08093940104C0109251
:1026B000CB011092F90181E0809393010895DC0130
:1026C000E0919301EE23E1F79E2F8C91882359F03E
:1026D000FD01A0EEB1E081918D939F5F8081882301
:1026E00011F09931C0F3E92FFF27E052FE4F10821D
:1026F000973048F081E08093CB011092F90183E09C
:102700008093940104C01092CB011092F90181E0F2
:10271000809393010895893128F4E82FFF27E05230
:10272000FE4F60830895089590E0E0EEF1E080E2CE
:1027300081939F5F9931D8F308958093960108950E
:10274000909193019923E1F76093CB019093F90164
:102750008093930108951092950108950F931F930C
:10276000CF93C82F80915401882321F00E949413A5
:1027700010925401809153010E94C717182F082FFF
:102780000F70005D12951F70105D63E480E00E9481
:102790008B1364E581E00E948B1362E582E00E9466
:1027A0008B1360E283E00E948B13612F84E00E9410
:1027B0008B13602F85E00E948B1360E081E00E9404
:1027C000A013C43021F4809153018F5F05C0C53040
:1027D00029F48091530181508093530180915301DA
:1027E0008F3F11F41092530180915301803118F002
:1027F0008FE080935301809153018F708093E700A5
:10280000C13029F4C09354018CE590E002C08DE5FD
:1028100090E0CF911F910F91089580E00E9458148D
:102820008FE08093E70087EB8093E50087E080935B
:10283000E60080EC8093E4008091E400886080935F
:10284000E400109293010895E82F20E030E0663014
:1028500070F58A52813558F4E13608F0EF7DEA527E
:10286000FF27EE0FFF1FE352F74F25913491A62F5C
:10287000BB27A0FF02C05FE001C050EF6695E62FC6
:10288000FF27E453FE4F40E0922F9F7084E036957F
:1028900027958A95E1F7A0FF02C09295907F8081ED
:1028A0008523892B808335964F5F443068F30895E4
:1028B00081118FEF90E0ECECF1E081939F5F943118
:1028C000E0F308951F920F920FB60F921124DF923A
:1028D000EF92FF920F931F932F933F934F935F932A
:1028E0006F937F938F939F93AF93BF93CF93EF9308
:1028F000FF93DD2480919901882361F480919701F1
:102900008F5F80939701843028F081E08093990154
:10291000D092970180915E01833071F4809198018B
:102920008F5F80939801813148F081E080935E0150
:102930008FE08093980102C0109298018091550118
:102940008150809355019091CB01992371F0882398
:1029500071F480919401882321F481E080939301A4
:1029600006C081508093940102C09093F901FF2426
:1029700090919301913009F056C080919501853076
:1029800010F4EF2C01C0E92EC0E000E010E08091CF
:10299000F901992787FD9095800F911F97FD17C02A
:1029A000FF20A9F48091F901E82FFF27E7FDF095BA
:1029B000E052FE4FE00FF11F8081DF2C87FF02C045
:1029C00091E0D92E8F7721F4FC2EF39401C080E2A0
:1029D000DD2029F0EE2019F06C2F80E201C06C2F71
:1029E0000E942414CF5F0F5F1F4FC63080F2C0E0FB
:1029F000ACEEB0E0ECECF1E081918D93CF5FC431AF
:102A0000D8F380919601811181E08093F40081E0F8
:102A1000F81611F48AEF03C08091F9018F5F80935B
:102A2000F9011092930180915501882319F483E0F4
:102A300080935501809195018A3019F41092950187
:102A400003C08F5F80939501FF91EF91CF91BF916C
:102A5000AF919F918F917F916F915F914F913F9136
:102A60002F911F910F91FF90EF90DF900F900FBE6D
:102A70000F901F901895CF93DF93CDB7DEB72297B5
:102A80000FB6F894DEBF0FBECDBFDC0149835A8379
:102A900020E02617B8F4FD01E20FF11DE081F89463
:102AA000F999FECF89819A8192BD81BDE0BDFA9AE4
:102AB000F99A789489819A81019689839A832F5F04
:102AC000261748F322960FB6F894DEBF0FBECDBF8F
:102AD000DF91CF910895CF93DF93CDB7DEB72297E3
:102AE0000FB6F894DEBF0FBECDBFDC0149835A8319
:102AF00020E02617B0F4FD01E20FF11DF894F999DA
:102B0000FECF89819A8192BD81BDF89A789480B573
:102B1000808389819A81019689839A832F5F261702
:102B200050F322960FB6F894DEBF0FBECDBFDF91F3
:102B3000CF91089585B18F6085B984B1876084B9DC
:102B400081E08DBD8CE58CBD08958EBD0DB407FE72
:102B5000FDCF8EB599270895289A289887E50E9479
:102B6000A51580E00E94A515482F5527CA01887336
:102B7000907023E0959587952A95E1F79927FC01B8
:102B8000E75BF64F24912093FA01FC01E80FF91F4F
:102B9000EF5AF64F859194919093FC018093FB013D
:102BA000CA010895CF93DF93EC01289A28986130E9
:102BB00009F583E50E94A5152091FA0180E190E0D6
:102BC000821B91099E0102C0369527958A95E2F7EE
:102BD000C9010E94A5158091FA019927089702C0A2
:102BE000CC0FDD1F8A95E2F78C2F0E94A51580E09F
:102BF0000E94A515289A28980E94AC1587FFFCCF43
:102C0000DF91CF910895CF93DF93EB0190E3289A62
:102C100028988130A1F484E50E94A51580E00E94E7
:102C2000A5158D2F99270E94A5158C2F0E94A515FB
:102C300080E00E94A51580E00E94A515982F892F9D
:102C40009927DF91CF910895EF92FF920F931F93F1
:102C5000CF93DF93EB017A018901289A289881307C
:102C6000F9F484E50E94A51580E00E94A5158D2F3A
:102C700099270E94A5158C2F0E94A51580E00E941F
:102C8000A515C0E0D0E0CE15DF0550F480E00E942D
:102C9000A515F80181938F012196CE15DF05B0F3BC
:102CA000DF91CF911F910F91FF90EF900895CF93F7
:102CB000DF93EB01289A2898813069F484E80E9418
:102CC000A51580E00E94A5158D2F99270E94A515B6
:102CD0008C2F0E94A515DF91CF9108951F93CF935C
:102CE000DF93EB01142F289A2898813081F484E82F
:102CF0000E94A51580E00E94A5158D2F99270E949E
:102D0000A5158C2F0E94A515812F0E94A515DF9176
:102D1000CF911F910895EF92FF920F931F93CF933E
:102D2000DF93EB017A018901289A28988130D9F440
:102D300084E80E94A51580E00E94A5158D2F992793
:102D40000E94A5158C2F0E94A515C0E0D0E0CE15DD
:102D5000DF0548F4F80181918F010E94A5152196A5
:102D6000CE15DF05B8F3DF91CF911F910F91FF9042
:102D7000EF900895CF93DF93EB01289A2898813044
:102D800009F583E80E94A5152091FA0180E190E001
:102D9000821B91099E0102C0369527958A95E2F71C
:102DA000C9010E94A5158091FA019927089702C0D0
:102DB000CC0FDD1F8A95E2F78C2F0E94A51580E0CD
:102DC0000E94A515289A28980E94AC1587FFFCCF71
:102DD000DF91CF910895EF92FF920F931F938C0193
:102DE0007B01289A289888E60E94A5152091FA016F
:102DF00080E190E0821B9109980102C036952795E9
:102E00008A95E2F7C9010E94A5158091FA019927D8
:102E1000089702C0000F111F8A95E2F78F2D99279E
:102E2000800F0E94A5158E2D0E94A51580E00E949E
:102E3000A51580E00E94A51580E00E94A51580E000
:102E40000E94A5151F910F91FF90EF90089527986C
:102E50002698249885B1806D85B91DB88EB18C6097
:102E60008EB98CE080936B0080ED80936C0080ECD9
:102E70008CBB8DBB0E94140B8093FD0108951F92A3
:102E80000F920FB60F9211242F933F934F935F939E
:102E90006F937F938F939F93AF93BF93EF93FF9322
:102EA0000E948717FF91EF91BF91AF919F918F91F2
:102EB0007F916F915F914F913F912F910F900FBE36
:102EC0000F901F9018951F920F920FB60F9211241A
:102ED0002F933F934F935F936F937F938F939F9322
:102EE000AF93BF93EF93FF930E948717FF91EF91EA
:102EF000BF91AF919F918F917F916F915F914F9112
:102F00003F912F910F900FBE0F901F90189523B1F6
:102F10002095207D8CB180958C70282B822F99274D
:102F200086FF02C094E011C027FF02C095E00DC0EB
:102F300082FF02C093E009C083FF02C092E005C097
:102F400084FF02C091E001C090E0992379F0809164
:102F50009901882359F080919B01882329F490934B
:102F60009A0181E080939B011092990180EC8CBBC7
:102F7000109289010895F89480919B01882321F093
:102F800080919A0110929B01789499270895282F97
:102F900080E02A3020F08F5F2A502A30E0F799270E
:102FA00034E0880F991F3A95E1F7282B822F992753
:102FB000089520E030E0843628F02F5F3F4F84569C
:102FC0008436D8F754E0220F331F5A95E1F78A3040
:102FD00028F02F5F3F4F8A508A30D8F744E0220F05
:102FE000331F4A95E1F79927282B392BC9010895FA
:102FF00080937C0083E880937A000E9400180895F3
:1030000040E050E08B9A839A80917A0080688093A8
:103010007A0080917A00806480937A0080917A00AF
:1030200084FFFCCF30E080917A00806480937A0046
:1030300080917A0084FFFCCF209178008091790004
:103040009927982F8827820F911D480F591F3F5F9E
:10305000383048F383E0559547958A95E1F78B988A
:10306000839880917A008F7780937A00CA010895BF
:103070009F92AF92BF92CF92DF92EF92FF920F9307
:103080001F93CF93DF93C0E0D0E099240E940018F3
:103090009C0180917C00882309F099C080915A019D
:1030A000833009F04CC083E02B3238078CF0AE013E
:1030B000FA01E552F64F859194918217930730F407
:1030C00093944E5F5F4F99E1991590F76DE216C0AA
:1030D000E3E020323E078CF4E92DFF27EE0FFF1FBF
:1030E000EF59F64F859194912817390720F493945E
:1030F000F3E6F91588F76BE201C060E281E00E9417
:103100008B13892D0E94C7179FE0A92EA82220E3C8
:10311000A20E182F12951F70120F60E280E00E941D
:103120008B13612F82E00E948B136A2D83E00E9433
:103130008B136AE284E00E948B1363E440C1843005
:1031400009F044C1E92DFF27EE0FFF1FE750F64FAE
:10315000859194918217930720F093948DE88915B7
:1031600088F7892D0E94D917EC0193E6991560F430
:103170006BE280E00E948B138D2F992787FD9A9533
:10318000182F105D612F05C060E280E00E948B1354
:103190006BE281E00E948B131FE0A12EAC22E0E3E2
:1031A000AE0EB4E0D595C795BA95E1F78C2F8F7028
:1031B0008E0F682F82E00E948B136A2D83E00E949D
:1031C0008B136AE284E00E948B1366E4F8C080915E
:1031D0007C00813009F0BEC0E90182E00E94F8174E
:1031E0000E9400189C01E92DFF27EE0FFF1FED5EE6
:1031F000F44F859194918217930720F49394F6E10C
:10320000F91588F7992029F486EF98E2A4E3B0E451
:1032100019C025E1291528F48AEB99E4ACE3B0E460
:1032200011C0292D3327220F331F220F331F235C98
:10323000344FF901E590F490F9013296059114911B
:10324000D801C7018093560190935701A09358016C
:10325000B0935901F1E09F2E90927C00CE01AA27F5
:1032600097FDA095BA2FBC01CD010E94CF1A7B011A
:103270008C018091560190915701A0915801B09115
:1032800059019C01AD01C801B7010E94181BDC0166
:10329000CB0120E030E040E85AE3BC01CD010E94C0
:1032A000181BDC01CB0120E030E040EC50E4BC0115
:1032B000CD010E94181B7B018C010E94B21A5B0198
:1032C0006C01862F9927AA2797FDA095BA2FBC01DC
:1032D000CD010E94CF1ADC01CB019C01AD01C801D8
:1032E000B7010E946F1ADC01CB0120E030E048EC0E
:1032F00052E4BC01CD010E94181BDC01CB01BC01D2
:10330000CD010E94B21A7B018C018A2D0E94C71741
:10331000A82EFFE0AF2220E3A20E8E2D0E94C71739
:10332000182F12951F70105D60E280E00E948B13D1
:1033300060E2892D0E948B1360E282E00E948B1371
:103340006A2D83E00E948B1366E584E00E948B1354
:10335000612F35C0C0917C00C230C1F580917900E9
:103360000E94C71780917800982F9F70E0E3AE2EDF
:10337000A90EE9E3EA1518F477E3A72EA90E682F42
:1033800062956F70162F105D1A3308F0195F61E4B3
:10339000892D0E948B1364E481E00E948B1363E407
:1033A0008C2F0E948B1380917900805D682F83E0C1
:1033B0000E948B13612F84E00E948B136A2D85E09D
:1033C0000E948B1360E086E00E948B13DF91CF9107
:1033D0001F910F91FF90EF90DF90CF90BF90AF9033
:1033E0009F900895CF93C82F60915B01662351F0A1
:1033F00010925B0180E00E94F81788E398E10E9438
:10340000E00A03C081E00E94A013C33051F488E3B6
:1034100098E10E94FF0A81E080935B018CE390E0D9
:1034200016C0C43039F480915A01843049F0C093F9
:103430005A010BC0C53049F480915A01843011F40F
:1034400083E001C084E080935A018DE390E0CF9146
:103450000895CF93C82F60915C01662351F01092BC
:103460005C0181E00E94F81788E398E10E94E00A7D
:1034700003C081E00E94A013C33051F488E398E1B7
:103480000E94FF0A81E080935C0186E490E002C024
:1034900087E490E0CF910895CF93C82F60915D01AC
:1034A000662351F010925D0182E00E94F81788E3D4
:1034B00098E10E94E00A03C081E00E94A013C3309B
:1034C00051F488E398E10E94FF0A81E080935D0156
:1034D00080E590E002C081E590E0CF9108955058DA
:1034E000192E84D001D06AC0BA1762077307840707
:1034F0009507B1F188F40EF410940B2EBA2FA02D7D
:10350000062E622F202D072E732F302D082E842F8C
:10351000402D092E952F502DFF275523B9F0591B0B
:1035200049F0573E98F0469537952795A795F04076
:103530005395C9F776F0BA0F621F731F841F30F4DA
:10354000879577956795B795F040939517FA0F2E65
:103550000895BF1BBB27BA0B620B730B840BF6CF0E
:10356000DEF660C097FB4ED09F3738F0FEE9F91BBE
:10357000982F872F762F6B2F05C051C09695879572
:1035800077956795F150D0F73EF4909580957095BA
:1035900061957F4F8F4F9F4F0895E89403C097FB2D
:1035A0000EF4F3DFB62F672F782F892F9EE90024C2
:1035B00005C09A95BB0F661F771F881F112499239A
:1035C000A1F08823B2F79F3F59F0BB0F48F421F4D4
:1035D000002011F460FF04C06F5F7F4F8F4F9F4F3B
:1035E000881F9795879597F9089519C0052E092684
:1035F00007FA440F551F5F3F79F0AA27A51708F077
:1036000051E04795880F991F9F3F31F0BB27B917AD
:1036100008F091E0879508959F919F9157C0662784
:103620007727882799270895592F482F372F262F36
:10363000DDDF01D0C3CF992339F0552329F09F57FF
:103640005F57950F13F4CAF1EDCF91589F3FE1F307
:10365000A62F00241124BB2766275527F8E0A6953E
:1036600020F4020E131EB41F651F220F331F441FC8
:10367000551FFA95A1F7F8E0E72F7727F8E0E695D0
:1036800020F4130EB41F651F7A1F330F441F551FFC
:10369000AA1FFA95A1F7F82F8827F69520F4B40F02
:1036A000651F7A1F8E1F440F551FAA1FEE1FFF2391
:1036B000A1F788231AF4939539F408C0000C111C63
:1036C000BB1F661F771F881F012808959FEF80EC9E
:1036D0000895AA1BBB1B51E107C0AA1FBB1FA61759
:1036E000B70710F0A61BB70B881F991F5A95A9F7AB
:0A36F00080959095BC01CD0108956E
:1036FA001E0101010101010101CB037B043E05CF3B
:10370A000564068A07A0070000500101001F1C1F5C
:10371A001E1F1E1F1F1E1F1E1F0C0102030405066B
:10372A000708090A0B0C0102030405060708090A1F
:10373A000B019E08A508AC08B308B908BF08010127
:0E374A000102010F01039A99394003010101A8
:00000001FF
